:020000040000FA
:0600000098EF16F012005B
:020006001200E6
:06000800B0EF02F012004F
:02000E000100EF
:0C0010004C2D000000010000CC0000009E
:04001C000F0E93161A
:1000200081169394939681948196F6D80F0E81163B
:10003000300E811227D815D90F0E8116300E81127D
:1000400021D80FD90F0E8116300E81121BD809D975
:100050000F0E8116818A16D8280EE66E17D8E55243
:10006000080EE66E13D8E552010EE66E0FD8E55283
:10007000060EE66E0BD8E5520F0EE66E07D8E55277
:1000800000D01200818612D981961200D9CFE6FFE6
:10009000E1CFD9FF10D9819481960F0E8116FE0E03
:1000A000DB50F00B8112EEDF0F0E8116FE0EDB38F7
:1000B000F00BF00B8112E6DF00D0E552E7CFD9FF5D
:1000C0001200D9CFE6FFE1CFD9FFF5D88184819620
:1000D0000F0E8116FE0EDB50F00B81128186E6D8E2
:1000E00081960F0E8116FE0EDB38F00BF00B81129D
:1000F0008186DCD8819600D0E552E7CFD9FF120087
:10010000D9CFE6FFE1CFD9FFFD0EDBCFF6FFFE0E24
:10011000DBCFF7FF0800F55011E0FD0EDBCFF6FF57
:10012000FE0EDBCFF7FF0800F550E66ECADFE552A2
:10013000FD0EDB2AFE0E01E3DB2AE6D700D0E552F6
:10014000E7CFD9FF1200D9CFE6FFE1CFD9FFFD0EEF
:10015000DBCFE9FFFE0EDBCFEAFFEF5010E0FD0E34
:10016000DBCFE9FFFE0EDBCFEAFFEF50E66EA9DF43
:10017000E552FD0EDB2AFE0E01E3DB2AE8D700D0B4
:10018000E552E7CFD9FF1200D9CFE6FFE1CFD9FF83
:10019000E652FE0EDB0404E1FD0EDB50800FDF6E45
:1001A000FE0EDB50020804E1FD0EDB50C00FDF6ED7
:1001B000DFCFE6FF6BDFE552E552E552E7CFD9FF2F
:1001C0001200D9CFE6FFE1CFD9FFE652E66AFE0E74
:1001D000DBCFE6FFD9DFE552E552DF6ADFCF00F083
:1001E000100EE76E0018E8AE02D0E73402D0E750F8
:1001F000005C06E2200EE66E64DFE552DF2AEED7F1
:10020000E66AFE0EDBCFE6FFBFDFE552E552E552C0
:10021000E552E7CFD9FF1200D9CFE6FFE1CFD9FFF2
:10022000020EE126DE6ADD6ADECF00F0DDCF01F0EE
:10023000D890015004E6100E005C270E015806E22B
:100240000000DF2A010E01E3DB2AEED700D0020E08
:10025000E15C02E2E16AE552E16EE552E7CFD9FFE7
:100260001200D9CFE6FFE1CFD9FF020EE126DE6A08
:10027000DD6ADECF00F0DDCF01F0D890015004E65A
:10028000C40E005C090E015806E20000DF2A010ED0
:1002900001E3DB2AEED700D0020EE15C02E2E16A64
:1002A000E552E16EE552E7CFD9FF120000000000F1
:1002B000000000001200D9CFE6FFE1CFD9FF020E07
:1002C000E126DE6ADD6ADECF00F0DDCF01F0D890F6
:1002D000015004E6E80E005C030E015806E200003F
:1002E000DF2A010E01E3DB2AEED700D0020EE15C2B
:1002F00002E2E16AE552E16EE552E7CFD9FF120072
:10030000D9CFE6FFE1CFD9FF81940F0E8116FE0E03
:10031000DB504009F00B8112C9DFB4DE0F0E8116ED
:10032000FE0EDB38F00BF00B8112C0DFABDE00D02D
:10033000E552E7CFD9FF12000000000000000000E6
:1003400000000000000000000000000000000000AD
:100350001200D9CFE6FFE1CFD9FFFB0EDBCF1DF0B6
:10036000FC0EDBCF1EF0FD0EDBCF1FF0FE0EDBCF51
:1003700020F02034000E201809E6D880000E1D540D
:10038000000E1E54000E1F54000E20540CE2D950D3
:10039000FB0FE96EFF0EDA20EA6EEE06000EEE5A53
:1003A000EE5AEE5ADAD7E552E7CFD9FF1200948E13
:1003B000949C200EAF6EAC8AAC84AC98AC9CAB8E97
:1003C000AB9CAB889E989E9A9D8AF28EF28C12000E
:1003D000D9CFE6FFE1CFD9FFE65200018751851959
:1003E00002E18851861901E1F8D785C0E9FF86C08E
:1003F000EAFF852B000E8623EFCFDFFF9C0E855D85
:10040000010E865904E35C0E856F010E866FDF5086
:1004100000D0E552E552E7CFD9FF1200D9CFE6FF71
:10042000E1CFD9FF020EE126DE6ADD6AACB210D060
:10043000DF2A010E01E3DB2AD9CFE9FFDACFEAFF99
:10044000100ED880EE54270EED5401E206D0EED700
:10045000FE0EDB50AD6E9EA8FED7020EE15C02E2FE
:10046000E16AE552E16EE552E7CFD9FF1200D9CF3C
:10047000E6FFE1CFD9FF030EE126FD0EDBCFDEFF65
:10048000DBCFDDFFA5DFE76E020EE7CFDBFFFC0E63
:10049000DB50F36E020EDB50F35C0DE0FD0EDBCFA4
:1004A000E9FFDB2AFE0EDBCFEAFF01E3DB2A020EC7
:1004B000DBCFEFFFE7D7FD0EDBCFE9FFFE0EDBCF93
:1004C000EAFFEF6ADECF00F0DDCF01F000C0F3FFFE
:1004D00001C0F4FF030EE15C03E200D0E16AE552E3
:1004E000E16EE552E7CFD9FF1200D9CFE6FFE1CFA9
:1004F000D9FF020EE126DE6ADD6AFD0EDBCFE9FFE1
:10050000FE0EDBCFEAFFEF5014E0FD0EDBCFE9FF7C
:10051000FE0EDBCFEAFFEF50E66E80DFE552DF2A0A
:10052000010E01E3DB2AFD0EDB2AFE0E01E3DB2ACE
:10053000E4D7010EF36EF46A020EE15C03E200D030
:10054000E16AE552E16EE552E7CFD9FF12000D0EE8
:10055000E66E64DFE5520A0EE66E60DFE5521200D9
:10056000DACFE4FFE2CFDAFFE9CFE4FFEACFE4FF3E
:10057000F6CFE4FFF7CFE4FFF5CFE4FFF3CFE4FFDE
:10058000F4CFE4FFFACFE4FF00EE18F0140EE80415
:1005900003E3EECFE4FFFBD700EE00F0180EE80413
:1005A00003E3EECFE4FFFBD7E6529EAA4DD01AEC50
:1005B00016F00001D76FAB50040B03E1AB50020BF8
:1005C00002E0AB98AB88ACA2FED781B205D0D7C011
:1005D000E6FF71EC16F0E552080E0001D75D0DE163
:1005E000000EE76ED619E8AE02D0D63503D0E7503C
:1005F000D880D65501E2D60727D00D0ED75D17E07B
:10060000400EE76ED619E8AE02D0E73402D0E750CC
:10061000D65D0DE2D651D62BE96EEA6AE9BEEA68EC
:100620005C0EE926010EEA22D7C0EFFF0DD0D6C03E
:10063000E9FFEA6AE9BEEA685C0EE926010EEA22F1
:10064000EF6AD66B010E846F9EA40AD0BECFAAF0CB
:10065000BFCFABF00001AC6BAD6B9785CD909E9496
:10066000E55200EE17F0180EE80403E3E5CFEDFFC6
:10067000FBD700EE2BF0140EE80403E3E5CFEDFF0B
:10068000FBD7E5CFFAFFE5CFF4FFE5CFF3FFE5CFEA
:10069000F5FFE5CFF7FFE5CFF6FFE5CFEAFFE5CFC2
:1006A000E9FFE5CFDAFF1100D9CFE6FFE1CFD9FFAF
:1006B0000A0EE12600014B0E826F010E836FFC0EC5
:1006C000DBCF00F0010EE76E0018E8AE02D0003478
:1006D00003D0E750D880005401E2E6D0FC0EDB5096
:1006E00028E1FD0EDBCF00F0FE0EDBCF01F0060EA1
:1006F00000C0DBFF070E01C0DBFF080EDB6A090E3E
:10070000DB6A82C0E6FF83C0E6FFD950060FE96EC0
:10071000DACFEAFFEECFE6FFEECFE6FFEECFE6FF61
:10072000EFCFE6FF7BEC13F0006E060EE15E0050AB
:1007300010D082C0E6FF83C0E6FFFD0EDBCFE6FFF0
:10074000FE0EDBCFE6FFE1EC12F0E552E552E5529A
:10075000E552000197AD84D04B0EE66E010EE66EB9
:10076000E8EC15F0E552E552020EF3CFDBFF030E85
:10077000F4CFDBFFDE6ADD6ADECF00F0DDCF01F013
:10078000020EDBCF02F0030EDBCF03F00250005C61
:10079000035001582EE2020EDBCF02F0030EDBCF36
:1007A00003F0DE50025CE96EDD500358EA6EE906A4
:1007B000000EEA5A4B0EE926010EEA22EF50E66ED1
:1007C000FC0EDB50040F006E016A00BE0168DE50B3
:1007D000005CE96EDD500158EA6E4B0EE926010E11
:1007E000EA22E552E750EF6EDF2A010E01E3DB2A31
:1007F000C3D7DE6ADD6ADECF00F0DDCF01F0FC0E8C
:10080000DB50050F046E056A04BE0568020EDB505E
:10081000045C026E030EDB500558036E0250005C50
:10082000035001581DE2000197A90BD0DECFE9FF6C
:10083000DDCFEAFF4B0EE926010EEA22300EEF6E05
:100840000AD0DECFE9FFDDCFEAFF4B0EE926010E2D
:10085000EA22200EEF6EDF2A010E01E3DB2ACBD75E
:10086000FC0EDB50050FE96EEA6AE9BEEA684B0E42
:10087000E926010EEA22EF6A000197AF08D082C094
:10088000E6FF83C0E6FF5FDCE552E5520DD082C093
:10089000E6FF83C0E6FF29DEE552E552020EF3CF04
:1008A000DBFF030EF4CFDBFF0A0EE15C02E2E16A3C
:1008B000E552E16EE552E7CFD9FF1200D9CFE6FF4E
:1008C000E1CFD9FF0C0EE126F80EDBCF02F0000ECF
:1008D000E76E0218E8AE02D0023403D0E750D880A9
:1008E000025402E3070E12D0F80EDBCF03F0160E0F
:1008F000E76E0318E8AE02D0033403D0E750D88087
:10090000035402E2170E02D0F80EDB28006E016AD3
:1009100000BE0168060E00C0DBFF070E01C0DBFF52
:10092000DE6ADD6AFB0EDBCF00F0FC0EDBCF01F0F0
:10093000FD0EDBCF02F0FE0EDBCF03F0226A236A4E
:10094000246A256A00C01DF001C01EF002C01FF01D
:1009500003C020F0FDEC11F0010A33E1F90EDBCF0A
:10096000E9FFDB2AFA0EDBCFEAFF01E3DB2A2D0EDB
:10097000EF6EFB0EDBCF00F0FC0EDBCF01F0FD0EC7
:10098000DBCF02F0FE0EDBCF03F0226A236A800E7B
:10099000246EBF0E256E00C01DF001C01EF002C007
:1009A0001FF003C020F021EC11F0FB0E1DC0DBFF97
:1009B000FC0E1EC0DBFFFD0E1FC0DBFFFE0E20C0C5
:1009C000DBFFFB0EDBCF00F0FC0EDBCF01F0FD0EFA
:1009D000DBCF02F0FE0EDBCF03F0226A236A246A2B
:1009E000256A00C01DF001C01EF002C01FF003C048
:1009F00020F0F4EC11F0010A49E1FB0EDBCF00F02E
:100A0000FC0EDBCF01F0FD0EDBCF02F0FE0EDBCFE4
:100A100003F0226A236A800E246E3F0E256E00C00A
:100A20001DF001C01EF002C01FF003C020F0FDEC5D
:100A300011F0010A2BE1006A016A200E026E410EDC
:100A4000036ED950FB0FE96EFF0EDA20EA6EEECF8F
:100A50001DF0EECF1EF0EECF1FF0EFCF20F000C064
:100A600022F001C023F002C024F003C025F021ECE5
:100A700011F020C0EDFF1FC0EDFF1EC0EDFF1DC037
:100A8000EFFFDF06010E01E2DB06B7D7FB0EDBCF7F
:100A900000F0FC0EDBCF01F0FD0EDBCF02F0FE0E0E
:100AA000DBCF03F0226A236A200E246E410E256EEE
:100AB00000C01DF001C01EF002C01FF003C020F0F6
:100AC000FDEC11F0010A2DE0FB0EDBCF00F0FC0E77
:100AD000DBCF01F0FD0EDBCF02F0FE0EDBCF03F02B
:100AE000226A236A200E246E410E256E00C01DF07E
:100AF00001C01EF002C01FF003C020F0CEEC10F0C9
:100B0000FB0E1DC0DBFFFC0E1EC0DBFFFD0E1FC079
:100B1000DBFFFE0E20C0DBFFDF2A010E01E3DB2A34
:100B2000B5D7DECF00F0DDCF01F0D950060FE96E6A
:100B3000DACFEAFF0050EE260150ED22010EF36EEF
:100B4000020EF3CFDBFF030EDB6A020EDBCF1EF0DB
:100B5000030EDBCF1FF009EC10F0080E1DC0DBFF09
:100B6000090E1EC0DBFF0A0E1FC0DBFF0B0E20C0EC
:100B7000DBFF020EDBCF00F0030EDBCF01F0060E31
:100B8000DBCF02F0070EDBCF03F001500318E8AE15
:100B900002D0033404D00250005C035001582EE20E
:100BA000080EDBCF00F0090EDBCF01F00A0EDBCF21
:100BB00002F00B0EDBCF03F0226A236A200E246EB4
:100BC000410E256E00C01DF001C01EF002C01FF0D6
:100BD00003C020F0CEEC10F0080E1DC0DBFF090EA4
:100BE0001EC0DBFF0A0E1FC0DBFF0B0E20C0DBFFA9
:100BF000020EDB2A030E01E3DB2ABBD7080EDBCF94
:100C000004F0090EDBCF05F00A0EDBCF06F00B0E69
:100C1000DBCF07F0226A236A246A400E256E04C0E7
:100C20001DF005C01EF006C01FF007C020F0CEEC7E
:100C300010F01DC000F01EC001F01FC002F020C067
:100C400003F0D950FB0FE96EFF0EDA20EA6EEECF0B
:100C50001DF0EECF1EF0EECF1FF0EFCF20F000C062
:100C600022F001C023F002C024F003C025F038ECCC
:100C700010F020C0EDFF1FC0EDFF1EC0EDFF1DC036
:100C8000EFFFFB0EDBCF00F0FC0EDBCF01F0FD0E23
:100C9000DBCF02F0FE0EDBCF03F0226A236A200EC8
:100CA000246E410E256E00C01DF001C01EF002C072
:100CB0001FF003C020F0FDEC11F0010A12E0FB0E62
:100CC000DB6AFC0EDB6A800EF36EFD0EF3CFDBFFFA
:100CD0003F0EF36EFE0EF3CFDBFFDF2A010E01E3C2
:100CE000DB2ADECF00F0DDCF01F00001800E011421
:100CF00059E0F90EDBCFE9FFDB2AFA0EDBCFEAFF82
:100D000001E3DB2A300EEF6EF90EDBCFE9FFDB2AC1
:100D1000FA0EDBCFEAFF01E3DB2A2E0EEF6E060EA2
:100D2000DBCF00F0070EDBCF01F0800E011410E0E6
:100D3000DECF02F0DDCF03F0060EDB50025C006E6A
:100D4000070EDB500358016E00C0DEFF01C0DDFF5F
:100D5000020EDB68030EDB68020EDBCF00F0030E31
:100D6000DBCF01F0DECF02F0DDCF03F0035001183E
:100D7000E8AE02D0013404D00050025C01500358A8
:100D800011E2F90EDBCFE9FFDB2AFA0EDBCFEAFF37
:100D900001E3DB2A300EEF6E020EDB06030E01E2EA
:100DA000DB06DAD7020EDB6A030EDB6A020EDBCF4C
:100DB00000F0030EDBCF01F0060EDBCF02F0070ED2
:100DC000DBCF03F001500318E8AE02D0033404D0A7
:100DD0000250005C0350015801E3ABD0FB0EDBCFA7
:100DE0001DF0FC0EDBCF1EF0FD0EDBCF1FF0FE0E64
:100DF000DBCF20F08EEC11F0040E1EC0DBFF050EE1
:100E00001FC0DBFF300EE76E040EDBCF00F0050ED7
:100E1000DBCF01F0E7500026000E0122F90EDBCFF8
:100E2000E9FFDB2AFA0EDBCFEAFF01E3DB2A00C091
:100E3000EFFF020EDBCF00F0030EDBCF01F0DF503F
:100E4000001803E1DE52DD5001180BE1F90EDBCF93
:100E5000E9FFDB2AFA0EDBCFEAFF01E3DB2A2E0EE5
:100E6000EF6E040EDBCF1EF0050EDBCF1FF009EC9A
:100E700010F0080E1DC0DBFF090E1EC0DBFF0A0EBE
:100E80001FC0DBFF0B0E20C0DBFF1DC000F01EC02B
:100E900001F01FC002F020C003F0D950FB0FE96E33
:100EA000FF0EDA20EA6EEECF1DF0EECF1EF0EECF91
:100EB0001FF0EFCF20F000C022F001C023F002C0ED
:100EC00024F003C025F037EC10F020C0EDFF1FC068
:100ED000EDFF1EC0EDFF1DC0EFFF006A016A200E8E
:100EE000026E410E036ED950FB0FE96EFF0EDA2041
:100EF000EA6EEECF1DF0EECF1EF0EECF1FF0EFCF7B
:100F000020F000C022F001C023F002C024F003C092
:100F100025F021EC11F020C0EDFF1FC0EDFF1EC039
:100F2000EDFF1DC0EFFF020EDB2A030E01E3DB2AFB
:100F30003DD7F90EDBCFE9FFFA0EDBCFEAFFEF6A10
:100F40000C0EE15C02E2E16AE552E16EE552E7CFA8
:100F5000D9FF1200D9CFE6FFE1CFD9FF060EE12677
:100F60000001979DFB0EDBCF1DF0FC0EDBCF1EF0CA
:100F7000FD0EDBCF1FF0FE0EDBCF20F0BDEC11F03D
:100F80001CC0DEFF1DC0DEFF1EC0DEFF1FC0DDFF78
:100F9000DD52DD52FB0EDBCF04F0FC0EDBCF05F0A3
:100FA000FD0EDBCF06F0FE0EDBCF07F0F90EDBCF38
:100FB0001EF0FA0EDBCF1FF009EC10F01DC008F098
:100FC0001EC009F01FC00AF020C00BF008C022F0BC
:100FD00009C023F00AC024F00BC025F004C01DF0A6
:100FE00005C01EF006C01FF007C020F021EC11F074
:100FF0001DC000F01EC001F01FC002F020C003F0B1
:10100000F90EDBCF14F0FA0EDBCF15F0166A176A73
:1010100015AE02D01668176814C01CF015C01DF07C
:1010200016C01EF017C01FF0DFCF21F0010EDBCF7E
:1010300022F0020EDBCF23F0030EDBCF24F097EC7F
:1010400015F018C010F019C011F01AC012F01BC032
:1010500013F010C01CF011C01DF012C01EF013C020
:101060001FF01EEC10F01DC00CF01EC00DF01FC0D4
:101070000EF020C00FF00CC022F00DC023F00EC007
:1010800024F00FC025F000C01DF001C01EF002C00A
:101090001FF003C020F037EC10F08EEC11F0040EBE
:1010A0001EC0DBFF050E1FC0DBFF000EE66E010E4B
:1010B000E66ED9CFE9FFDACFEAFFEECFE6FFEECF5B
:1010C000E6FFEECFE6FFEFCFE6FF7BEC13F0006E1E
:1010D000060EE15E0050000197AF09D0000EE66EEB
:1010E000010EE66EA3EC00F0E552E5520CD0000EC6
:1010F000E66E010EE66E75EC02F0E552E552F3CFB6
:10110000A4F0F4CFA5F0000197AF06D02E0EE66E46
:1011100061EC00F0E55205D02E0EE66E0EEC02F00A
:10112000E552E66A040EDBCFE6FF050EDBCFE6FFF5
:1011300054EC03F0E552E552E552060EE15C02E2A2
:10114000E16AE552E16EE552E7CFD9FF1200D9CF4F
:10115000E6FFE1CFD9FFE652800EDF6EDF500008D8
:1011600013E2FE0EDB50DF1406E0310EE66E0EECED
:1011700002F0E55205D0300EE66E0EEC02F0E552BC
:10118000DF407F0BDF6EEAD7E552E552E7CFD9FFAC
:101190001200D9CFE6FFE1CFD9FF020EE126FE0E05
:1011A000DB50F00BE8380F0B300FDF6EDF503908E3
:1011B00003E2070EDF24DF6EFE0EDB500F0B300F55
:1011C000E76E010EE7CFDBFFDB5039080AE2070EBE
:1011D000006E010EDBCFE7FF0050E726010EE7CFE0
:1011E000DBFFDFCFE6FF0EEC02F0E552010EDBCFB6
:1011F000E6FF0EEC02F0E552680EE66E0EEC02F031
:10120000E552020EE15C02E2E16AE552E16EE5526E
:10121000E7CFD9FF1200816A936A939093929394D7
:1012200093969398939A939C938E816AC26A070EC1
:10123000C16E926E1F0E896E8268860E946E9490B7
:101240009492948494969498949A949C948E120078
:101250000001BA6BBB6BBC6BBD6BAA6BAB6BAC6BB1
:10126000AD6B000EE66EE66A55EC16F0E552E552FF
:101270008986899689869E90CD809EA005D00001A2
:10128000BC2B000EBD239E9082B4F7D7CD901200E8
:10129000C2DF8998100EE66E270EE66EE66AE66AF1
:1012A000A9EC01F0E552E552E552E5520EEC00F0F2
:1012B000010EE66E46EC00F0E552100EE66E270ECB
:1012C000E66EE66AE66AA9EC01F0E552E552E552FF
:1012D000E552AAC1E6FFABC1E6FF80EC00F0E552A3
:1012E000E552C00EE66E46EC00F0E552ACC1E6FFFA
:1012F000ADC1E6FF80EC00F0E552E552900EE66EDF
:10130000D00EE66E030EE66EE66AA9EC01F0E55239
:10131000E552E552E552010EE66EE1EC00F0E552D1
:10132000AEC1E6FFAFC1E6FF80EC00F0E552E5524A
:10133000020EE66EE1EC00F0E552B0C1E6FFB1C18D
:10134000E6FF80EC00F0E552E552900EE66ED00E1E
:10135000E66E030EE66EE66AA9EC01F0E552E55290
:10136000E552E5528986D7EC01F00001979F0C0EFB
:10137000E66E0EEC02F0E552A00EE66E860EE66E0C
:10138000010EE66EE66AA9EC01F0E552E552E5527F
:10139000E5529EC100F09FC101F0026A00C0E6FF65
:1013A00001C0E6FF02C0E6FF40C1E6FF41C1E6FF23
:1013B000CFEC15F0036E050EE15E035040C1E6FF71
:1013C00041C1E6FF75EC02F0E552E552F3CFA4F01F
:1013D000F4CFA5F0A0C100F0A1C101F0026A00C0E5
:1013E000E6FF01C0E6FF02C0E6FF40C1E6FF41C1E3
:1013F000E6FFCFEC15F0036E050EE15E035040C131
:10140000E6FF41C1E6FF75EC02F0E552E552F3CF8D
:10141000A4F0F4CFA5F0A2C100F0A3C101F0026ACC
:1014200000C0E6FF01C0E6FF02C0E6FF40C1E6FFE4
:1014300041C1E6FFCFEC15F0036E050EE15E0350EF
:1014400040C1E6FF41C1E6FF75EC02F0E552E5520E
:10145000F3CFA4F0F4CFA5F0A00EE66E860EE66EF4
:10146000010EE66EE66AA9EC01F0E552E552E5529E
:10147000E552CD6ACD8ECD9ACD98CD96CD84CD92C4
:10148000CD909F80000EE66EE66A55EC16F0E552B0
:10149000E5529E90F28C9D90F29EF29C9484B19CB9
:1014A000040EBD6ED08E9D84F28E0001978F020EC9
:1014B000E66EE1EC00F0E552010EE66EE1EC00F0C4
:1014C000E552B2C1E6FFB3C1E6FF80EC00F0E552A1
:1014D000E552A00EE66E860EE66E010EE66EE66A38
:1014E000A9EC01F0E552E552E552E5520001979B67
:1014F000A26BA36BB26BB36BB46BB56BA9DED88078
:10150000660E0001AA55030EAB55000EAC55000E39
:10151000AD5504E2978B090EA26FA36B97A510D06F
:10152000AA0EE96E000EEA6EBA51EE24BA6FBB51F4
:10153000EE20BB6FBC51EE20BC6FBD51EE20BD6FE5
:10154000BA0EE96E000EEA6EB251EE24B26FB351DC
:10155000EE20B36FB451EE20B46FB551EE20B56FED
:10156000A22B000EA3230A0EA25D000EA359C6E310
:101570000B0EE66E010EE66EC4EC00F0E552E5528D
:10158000D880C00E0001B255210EB355000EB455DF
:10159000000EB55509E3700EB25D210EB359000E71
:1015A000B459000EB55920E2A6C100F0A7C101F060
:1015B000026A00C0E6FF01C0E6FF02C0E6FF40C1CC
:1015C000E6FF41C1E6FFCFEC15F0036E050EE15ECC
:1015D0000350C2C1E6FFC3C1E6FF80EC00F0E55254
:1015E000E5520001978B1ED0979BA4C100F0A5C1C6
:1015F00001F0026A00C0E6FF01C0E6FF02C0E6FF9C
:1016000040C1E6FF41C1E6FFCFEC15F0036E050EC9
:10161000E15E0350C4C1E6FFC5C1E6FF80EC00F007
:10162000E552E5520001979F000EE66E010EE66E50
:1016300075EC02F0E552E552F3CFA4F0F4CFA5F03B
:10164000090EE66E0EEC02F0E55240C1E6FF41C124
:10165000E6FFB2C0E6FFB3C0E6FFB4C0E6FFB5C028
:10166000E6FF7BEC13F0006E060EE15E005040C119
:10167000E6FF41C1E6FF75EC02F0E552E552F3CF1B
:10168000A4F0F4CFA5F0A7EC02F00001978FC00EF4
:10169000E66E46EC00F0E552BEC1E6FFBFC1E6FFD4
:1016A00080EC00F0E552E5520B0EE66E020EE66E9F
:1016B000C4EC00F0E552E55240C1E6FF41C1E6FF4F
:1016C000B2C0E6FFB3C0E6FFB4C0E6FFB5C0E6FFB8
:1016D0007BEC13F0006E060EE15E005040C1E6FFA9
:1016E00041C1E6FFA3EC00F0E552E552900EE66E34
:1016F000D00EE66E030EE66EE66AA9EC01F0E55246
:10170000E552E552E552020EE66EE1EC00F0E552DC
:10171000010EE66EE1EC00F0E552B4C1E6FFB5C1A2
:10172000E6FF80EC00F0E552E552C00EE66E46ECB6
:1017300000F0E552C6C1E6FFC7C1E6FF80EC00F04D
:10174000E552E5520001979FA8C100F0A9C101F040
:10175000026A00C0E6FF01C0E6FF02C0E6FF40C12A
:10176000E6FF41C1E6FFCFEC15F0036E050EE15E2A
:101770000350000EE66E010EE66E75EC02F0E552C7
:10178000E552F3CFA4F0F4CFA5F08998100EE66EE1
:10179000270EE66EE66AE66AA9EC01F0E552E5522C
:1017A000E552E55280B4FED7A7EC02F00001978F16
:1017B000020EE66EE1EC00F0E552010EE66EE1ECA1
:1017C00000F0E552BCC1E6FFBDC1E6FF80EC00F0D1
:1017D000E552E5520001979F230EE66E0EEC02F0F3
:1017E000E552090EE66E0EEC02F0E552AEC100F0D5
:1017F000AFC101F0026A00C0E6FF01C0E6FF02C00F
:10180000E6FF40C1E6FF41C1E6FFCFEC15F0036EF5
:10181000050EE15E0350000EE66E010EE66E75ECFD
:1018200002F0E552E552F3CFA4F0F4CFA5F0A7EC17
:1018300002F0000EE66EE66A39EC16F0E552E5526B
:101840009C0EB16EA092A192B1800001A26BA36B1D
:101850008998500EE66EC30EE66EE66AE66AA9EC5B
:1018600001F0E552E552E552E5520001BA6BBB6B5F
:10187000BC6BBD6BB26BB36BB46BB56BAA6BAB6B74
:10188000AC6BAD6B000EE66EE66A55EC16F0E552F9
:10189000E552898689968986CD809EA012D0AA0EAF
:1018A000E96E000EEA6E0001BA51EE24BA6FBB5128
:1018B000EE20BB6FBC51EE20BC6FBD51EE20BD6F62
:1018C0009E90A1A20DD0A1920001A22B000EA323F5
:1018D000320ED880A255000EA35502E2898802D0AC
:1018E00082B4DBD7B190000197A510D0AA0EE96EA3
:1018F000000EEA6EBA51EE24BA6FBB51EE20BB6FF8
:10190000BC51EE20BC6FBD51EE20BD6F978F080E0D
:10191000E66E010EE66EC4EC00F0E552E55289B8C1
:1019200009D0B8C1E6FFB9C1E6FF80EC00F0E5528E
:10193000E55208D0BAC1E6FFBBC1E6FF80EC00F07B
:10194000E552E552900EE66ED00EE66E030EE66EA0
:10195000E66AA9EC01F0E552E552E552E5520001D4
:10196000A26BA36BBE6BBF6BC06BC16BC26B240E53
:10197000C36FF40EC46FC56BBA6BBB6BBC6BBD6B36
:10198000AA6BAB6BAC6BAD6BB26BB36BB46BB56B83
:101990005FDC000197A520D3AA0EE96E000EEA6E67
:1019A000BA51EE24BA6FBB51EE20BB6FBC51EE2092
:1019B000BC6FBD51EE20BD6FBA0EE96E000EEA6E2F
:1019C000EE50BE5DEE50BF59EE50C059EE50C159B9
:1019D00008E2BAC0BEF0BBC0BFF0BCC0C0F0BDC022
:1019E000C1F0BA0EE96E000EEA6EC251EE5CC35150
:1019F000EE58C451EE58C551EE5808E2BAC0C2F0D4
:101A0000BBC0C3F0BCC0C4F0BDC0C5F0978F010E11
:101A1000E66E020EE66EC4EC00F0E552E552E66AB0
:101A2000A2C000F0A3C001F0090ED8800056000E3D
:101A3000015600C0E6FF01C0E6FF54EC03F0E5529A
:101A4000E552E5520001979FE66AA2C000F0A3C0EC
:101A500001F0090ED8800056000E015600C0E6FFC6
:101A600001C0E6FF54EC03F0E552E552E552090EE1
:101A7000E66E0EEC02F0E552000EE66E010EE66E2A
:101A8000BAC0E6FFBBC0E6FFBCC0E6FFBDC0E6FFD4
:101A90007BEC13F0006E060EE15E0050000EE66E69
:101AA000010EE66E75EC02F0E552E552F3CFA4F0BC
:101AB000F4CFA5F0BA0EE96E000EEA6E0001B25145
:101AC000EE24B26FB351EE20B36FB451EE20B46F79
:101AD000B551EE20B56F978F090EE66E020EE66ED9
:101AE000C4EC00F0E552E552000EE66E010EE66E23
:101AF000A3EC00F0E552E5520001A22B000EA32357
:101B0000090ED880A255000EA35501E361D2979F1C
:101B1000A7EC02F0B2C01CF0B3C01DF0B4C01EF0C0
:101B2000B5C01FF01CEC10F01DC000F01EC001F08D
:101B30001FC002F020C003F0226A236A200E246E28
:101B4000410E256E00C01DF001C01EF002C01FF046
:101B500003C020F0CEEC10F01DC0CAF01EC0CBF0C8
:101B60001FC0CCF020C0CDF0B2C0B6F0B3C0B7F00B
:101B7000B4C0B8F0B5C0B9F00A0E216E226A236A6B
:101B8000246AB6C01CF0B7C01DF0B8C01EF0B9C0C2
:101B90001FF0F6EC15F01CC0B6F01DC0B7F01EC06B
:101BA000B8F01FC0B9F089B83DD0290E046EDA0E26
:101BB000056E280E066E390E076ECAC022F0CBC025
:101BC00023F0CCC024F0CDC025F004C01DF005C02A
:101BD0001EF006C01FF007C020F021EC11F01DC060
:101BE00000F01EC001F01FC002F020C003F0DF0EA5
:101BF000226E4F0E236E0D0E246EBE0E256E00C09B
:101C00001DF001C01EF002C01FF003C020F038EC30
:101C100010F01DC0C6F01EC0C7F01FC0C8F020C025
:101C2000C9F03CD0180E046EB40E056E900E066E10
:101C3000380E076ECAC022F0CBC023F0CCC024F00F
:101C4000CDC025F004C01DF005C01EF006C01FF079
:101C500007C020F021EC11F01DC000F01EC001F003
:101C60001FC002F020C003F00A0E226ED70E236EB2
:101C7000230E246E3D0E256E00C01DF001C01EF027
:101C800002C01FF003C020F038EC10F01DC0C6F0F9
:101C90001EC0C7F01FC0C8F020C0C9F0000EE66E1D
:101CA000010EE66EB6C0E6FFB7C0E6FFB8C0E6FFBD
:101CB000B9C0E6FF7BEC13F0006E060EE15E00504B
:101CC0002A0EE66E0EEC02F0E552000EE66E010EF4
:101CD000E66E75EC02F0E552E552F3CFA4F0F4CFD6
:101CE000A5F0090EE66E0EEC02F0E5520001978FAA
:101CF000020EE66EE1EC00F0E552010EE66EE1EC5C
:101D000000F0E552B6C1E6FFB7C1E6FF80EC00F097
:101D1000E552E552070EE66E010EE66EC4EC00F0E9
:101D2000E552E552000EE66E010EE66EB6C0E6FF25
:101D3000B7C0E6FFB8C0E6FFB9C0E6FF7BEC13F022
:101D4000006E060EE15E0050000EE66E010EE66EBD
:101D5000A3EC00F0E552E5520001979F030EE66EFA
:101D6000000EE66E010EE66EC6C0E6FFC7C0E6FFD7
:101D7000C8C0E6FFC9C0E6FF5EEC04F0006E070EC7
:101D8000E15E0050000EE66E010EE66E75EC02F0AC
:101D9000E552E552F3CFA4F0F4CFA5F0200EE66EA5
:101DA0000EEC02F0E552000197AB0BD03F0EE66E51
:101DB0000EEC02F0E5523F0EE66E0EEC02F0E5523C
:101DC00017D089B806D06E0EE66E0EEC02F0E55222
:101DD00005D0750EE66E0EEC02F0E552460EE66E8C
:101DE0000EEC02F0E552090EE66E0EEC02F0E55242
:101DF0000001978F010EE66E020EE66EC4EC00F055
:101E0000E552E552000EE66E010EE66EA3EC00F020
:101E1000E552E5520A0EE66E020EE66EC4EC00F0E4
:101E2000E552E552000197AB0BD03F0EE66E61EC38
:101E300000F0E5523F0EE66E61EC00F0E55212D084
:101E400089B806D06E0EE66E61EC00F0E55205D062
:101E5000750EE66E61EC00F0E552460EE66E61EC42
:101E600000F0E5520001979FC20EE96E000EEA6E87
:101E7000EE50BE5D086EEE50BF59096EEE50C0596F
:101E80000A6EEE50C1590B6E08C01CF009C01DF05F
:101E90000AC01EF00BC01FF01CEC10F01DC004F0B7
:101EA0001EC005F01FC006F020C007F0226A236A9A
:101EB000C80E246E420E256E04C01DF005C01EF033
:101EC00006C01FF007C020F021EC11F01DC000F08B
:101ED0001EC001F01FC002F020C003F0CAC022F0F3
:101EE000CBC023F0CCC024F0CDC025F000C01DF045
:101EF00001C01EF002C01FF003C020F0CEEC10F0B5
:101F00001DC0C6F01EC0C7F01FC0C8F020C0C9F079
:101F10002B0EE66E0EEC02F0E5522D0EE66E0EEC88
:101F200002F0E552020EE66E000EE66E010EE66E5F
:101F3000C6C0E6FFC7C0E6FFC8C0E6FFC9C0E6FFEF
:101F40005EEC04F0006E070EE15E0050000EE66EDF
:101F5000010EE66E75EC02F0E552E552F3CFA4F007
:101F6000F4CFA5F0250EE66E0EEC02F0E55200016E
:101F7000B26BB36BB46BB56B900EE66ED00EE66EC3
:101F8000030EE66EE66AA9EC01F0E552E552E55271
:101F9000E5520001978F010EE66EE1EC00F0E5528C
:101FA000C0C1E6FFC1C1E6FF80EC00F0E552E5529A
:101FB00080B4FED7F40EE66E010EE66EE66AE66ABF
:101FC000A9EC01F0E552E552E552E55280A4FED7B6
:101FD000A7EC02F000019795A80EE66E610EE66E82
:101FE000E66AE66AA9EC01F0E552E552E552E552EF
:101FF00000010A0EA25D000EA35901E2C9D4A7ECAC
:0E20000002F00001A26BA36B83EF0BF0120045
:02200E00279E0B
:1020100008D0279E1FAE05D01E6C1F1EE86A1F2227
:10202000278E1FC019F01EC018F02B6A2A6A8E0E68
:102030001A6E1B6A77EF12F0279E0CD0279E1FAEF8
:1020400009D01C6C1D1E1E1E1F1EE86A1D221E22AA
:102050001F22278E1FC019F01EC018F01DC02BF0C4
:102060001CC02AF09E0E1A6E1B6A77EF12F0257EB6
:10207000276AB3EC12F0CBEC12F027B65BEF12F04C
:1020800027A20AD027AA03D027BE5BEF12F027A40D
:1020900067EF12F064EF12F027AA05D027AC67EFC4
:1020A00012F064EF12F027A00AD027A808D027BEAC
:1020B00004D027A402D070EF12F074EF12F02A6A55
:1020C0001B6A2550205C296E10E31DC02BF01EC03A
:1020D00018F01FC019F020C028F022C01DF023C046
:1020E0001EF024C01FF0273A09D022C02BF023C0D5
:1020F00018F024C019F025C028F0296C279E27BCB1
:10210000278E28C01AF027B0A3EF12F01A0E29600C
:10211000A3EF12F01A6A206A27A408D01D6C1E1EB5
:102120001F1E201EE86A1E221F22202227AC08D074
:102130002B6C181E191E1A1EE86A182219221A2260
:102140001C6A295207E020341F321E321D321C3215
:10215000292EF9D71D502B261E5018221F50192248
:1021600020501A221CC02AF0279E1AAE0BD02A6CCF
:102170002B1E181E191E1A1EE86A2B22182219225D
:102180001A22278E1AA006D0D880193218322B3284
:102190002A32282A28C01AF077EF12F0276AB3EC07
:1021A00012F0CBEC12F027B65BEF12F027A205D0AD
:1021B00027BA5BEF12F062EF12F027BA6EEF12F05F
:1021C00027A005D027B85BEF12F06EEF12F027B80A
:1021D00062EF12F01B6A7F0E20241A6EE86A1B223F
:1021E00025501A5EE86A1B5A1A0E286E206A2A6A5F
:1021F0002B6A186A196A22501D5E23501E5A2450F9
:102200001F5A000E205A09E722501D2623501E2275
:1022100024501F22000E202201D02A8AD8901D3679
:102220001E361F362036D8902A362B3618361936E9
:10223000282EE1D71F501E101D10D8A42A8A77EF30
:1022400012F0276AB3EC12F0CBEC12F027B65BEF7A
:1022500012F027A205D027B85BEF12F062EF12F060
:1022600027AA05D027B05BEF12F062EF12F027B07B
:1022700002D027A802D06EEF12F01B6A255020244E
:102280001A6EE86A1B227E0E1A5EE86A1B5A2A6AD8
:102290002B6A186A196A24501F02F4CF19F0F3CF81
:1022A00018F023501F02F3502B26F4501822000E72
:1022B000192224501E02F3502B26F4501822000E2F
:1022C000192222501F02F3502A26F4502B22000E0E
:1022D0001822192223501E02F3502A26F4502B22D2
:1022E000000E1822192224501D02F3502A26F45001
:1022F0002B22000E1822192222501E02F4502A26E8
:10230000000E2B221822192223501D02F4502A26D7
:10231000000E2B221822192277EF12F0276AB3EC55
:1023200012F027B698EF11F027A20ED027B405D0EF
:102330007F0E1F6EFF0E1E6E1FD0800E1F6E1E6A58
:102340001BD01F6A1E6A18D027B0FBD78F0E2060E3
:10235000EDD77E0E2064F5D78E0E205C05E0D89078
:102360001F321E32202AF8D727A406D01E6C1F1E4B
:10237000E86A1F221FAEE5D71200276AB3EC12F0FD
:1023800027B6C7EF11F027A20FD027B407D07F0ED2
:102390001F6EFF0E1E6E1D6E1C6E25D0800E1F6EF2
:1023A00001D01F6A000EF6D727B0FBD71C6A9F0E1C
:1023B0002060EBD77E0E2064F4D79E0E205C07E0F1
:1023C000D8901F321E321D321C32202AF6D727A485
:1023D0000AD01C6C1D1E1E1E1F1EE86A1D221E2216
:1023E0001F221FAEDED7120006EC12F027B6000C3B
:1023F00027B0000C27B4000C010C06EC12F027B635
:10240000000C27B0000C27A4000C010C276AB3ECC9
:1024100012F0CBEC12F027B6120027AE08D027A09E
:1024200004D027A802D02780120027901200255040
:10243000205C0BE124501F5C08E123501E5C05E189
:1024400022501D5C02E127801200D8A002D0278E06
:1024500010D0205025C020F0256E1F5024C01FF042
:10246000246E1E5023C01EF0236E1D5022C01DF08E
:10247000226E2550205C10E0FF0F09E0279027B462
:1024800003D027AE2784120027AE27941200252AF6
:10249000D89024322332223222501D5E23501E5AFD
:1024A00024501F5A1FBEEAD7D8901D361E361F363D
:1024B000202EF8D7C8D77F0E206EFF0E1F6E1E6E1F
:1024C0001D6E12007F0E27BEFF0E206E02D07F0E03
:1024D000206E800E1F6E1E6A1D6AF3D727AE04D0D1
:1024E000800E206E1F6AF7D7206A1F6AF4D7195032
:1024F00018102B102A10F8E01BBEF0D719BE0CD014
:102500001A501B10EBE0D8902A362B3618361936A5
:102510001A06D8A01B06F2D71B50D4E11A28D2E025
:102520002AAE11D07F0E2A1402E12BA00CD02B2A48
:10253000E86A1822192207E3D880193218322B32A0
:102540001A2A1A28BFE01A50C9E02BC01DF018C083
:102550001EF019341F6E1A30206E1F32209E27BEC7
:10256000208E61EF12F01F36203602E32784277E8B
:1025700006E12780206A1F6A1E6A1D6A1200202851
:1025800003E0D8801F321200D8901F3202E1278268
:102590001200278612002436253602E3278C277E78
:1025A00006E12788256A246A236A226A1200252800
:1025B00003E0D88024321200D8902432EAE1278A3E
:0225C000120007
:0E25C200D9CFE6FFDACFE6FFFA0EE3CFD9FF5E
:1025D000FB0EE3CFDAFFFD0EE35209E72D0EDE6EB0
:1025E000FC0EE31EE32AFD0ED8B4E306E31EE6521A
:1025F000E652E652FD0EE124E76EFF0EE220E46EA5
:10260000E652F70EE3CFE6FFF70EE3CFE6FF51EC1D
:1026100013F0F90EE124E96EFF0EE220EA6E41ECC0
:1026200013F00AE13EEC13F009E141EC13F008E18C
:102630003EEC13F007E108D04CEC13F047EC13F03C
:102640004CEC13F047EC13F04CEC13F0DE6AF90E8F
:10265000E126FF0EE222FF0EE3CFDAFFE552FF0E86
:10266000E3CFD9FFE552FC0EE124E96EFF0EE22034
:10267000EA6EEECFF3FFEFCFF4FF1200EF380F0B4F
:102680001200EF500F0B02E1EE52D8841200EF3827
:102690000F0B300FDE6E1200EE500F0B300FDE6EA0
:1026A0001200FC0EE3CFE9FFFD0EE3CFEAFF100EB0
:1026B000E66EEE6AEE6AEF6AD890FD0EE336FE0E25
:1026C000E336ED36ED36EF36FF0EE30609E072EC49
:1026D00013F0EE5272EC13F0EE5272EC13F0EDD7F1
:1026E000E56E1200030EEF24E8B6EF6E300EEF2415
:1026F000E8BEEF6E000CD9CFE6FFDACFE6FFF80EAA
:10270000E3CFD9FFF90EE3CFDAFFE652E652E65205
:10271000E652E652FB0EE124E76EFF0EE220E46E85
:10272000E652F30EE3CFE6FFF30EE3CFE6FFF30E40
:10273000E3CFE6FFF30EE3CFE6FF00EC14F0F50E77
:10274000E124E96EFF0EE220EA6EEDEC13F019E1F0
:10275000F0EC13F018E1EDEC13F017E1F0EC13F0EE
:1027600016E1EDEC13F015E1F0EC13F014E1EDECF3
:1027700013F013E1F0EC13F012E1EDEC13F011E1C2
:1027800012D0F6EC13F0FBEC13F0F6EC13F0FBECCC
:1027900013F0F6EC13F0FBEC13F0F6EC13F0FBEC9B
:1027A00013F0F6EC13F0FBEC13F0DE6AF50EE12605
:1027B000FF0EE222FF0EE3CFDAFFE552FF0EE3CF7A
:1027C000D9FFE552FA0EE124E96EFF0EE220EA6E2F
:1027D000EECFF3FFEFCFF4FF1200EF380F0B120034
:1027E000EF500F0B02E1EE52D8841200EF380F0BBE
:1027F000300FDE6E1200EE500F0B300FDE6E120047
:10280000FA0EE3CFE9FFFB0EE3CFEAFF200EE66E00
:10281000EE6AEE6AEE6AEE6AEF6AD890FB0EE33675
:10282000FC0EE336FD0EE336FE0EE336ED36ED36F6
:10283000ED36ED36EF36FF0EE3060FE02FEC14F029
:10284000EE522FEC14F0EE522FEC14F0EE522FEC6F
:1028500014F0EE522FEC14F0E1D7E56E1200030EE7
:10286000EF24E8B6EF6E300EEF24E8BEEF6E000CFA
:102870000010181C1E1C1810000103070F0703018D
:10288000040E1F0E0E0E0E0E0E0E0E0E0E1F0E045A
:1028900002040E111F100E0008040E111F100E006E
:1028A00008040E010F110F000205020000000000D5
:1028B0002E2E2E00506F727420636F6D6D20333892
:1028C000343030206F7576657274200D0A00696EA1
:1028D000746572666163652049434D373535352C23
:1028E00020513D32304D687A202C52656C616973FD
:1028F0002047616D6D652C204250207374617274A5
:10290000200D0A004331383A203138465F43617068
:102910006163696D5F49434D373535355F434350DA
:10292000315F32304D687A5F52533233325F4C43FD
:10293000445F3132303231372E630D0A004F4B2065
:102940004D65737572652043617061205A45524F21
:102950003D313030207046203A200050524F424CDA
:10296000454D4521204D6573757265204361706149
:102970005A65726F20313030704620494E535441B1
:10298000424C452120383630202B2D33203A200070
:10299000496E73657265722043782065742061709A
:1029A000707579657220737572204250207374615E
:1029B00072742000313846204361706163696D652F
:1029C00074726520006D6F6E6F737461622049438D
:1029D0004D373535350031706620757020746F20A5
:1029E0003230303075460076657273696F6E204CF8
:1029F00043442032303132005A65726F4368656358
:102A00006B3A202020202020002020496E73657220
:102A1000742043782020202020004D6F792E3D2007
:102A20002020202020202020202000656E206E61A4
:102A30006E6F46202000656E204D6963726F4620E0
:102A4000004D65737572653A2020202020202020DB
:102A5000200053746162696C6974653A20202020FB
:102A6000202000537461727420666F72204E657866
:102A7000742020002042414400204F4B2000417030
:0F2A8000707579657220425020535441525400B2
:102A90000E0EF66E000EF76E000EF86E00010900C5
:102AA000F550DF6F0900F550E06F03E1DF6701D0FB
:102AB0003DD00900F550DA6F0900F550DB6F0900D1
:102AC000F550DC6F09000900F550E96E0900F5507A
:102AD000EA6E090009000900F550DD6F0900F550A4
:102AE000DE6F09000900F6CFE1F0F7CFE2F0F8CF92
:102AF000E3F0DAC0F6FFDBC0F7FFDCC0F8FF00014F
:102B0000DD5302E1DE5307E00900F550EE6EDD070C
:102B1000F8E2DE07F9D7E1C0F6FFE2C0F7FFE3C055
:0E2B2000F8FF0001DF07000EE05BBFD71200D8
:022B2E001C5039
:102B30002102F3CF18F0F4CF19F02202F350192636
:102B4000000EF4201A6E1C502302F3501A26000EB9
:102B5000F4201B6E1C502402F3501B261D50210232
:102B6000F3501926F4501A22000E1B221D50220287
:102B7000F3501A26F4501B221D502302F3501B263B
:102B80001E502102F3501A26F4501B221E5022021E
:0E2B9000F3501B261F502102F3501B2612008B
:022B9E00FB0E2C
:102BA000E3CFF6FFFC0EE3CFF7FFFD0EE3CFF8FF18
:102BB000FE0EE3CFE9FFFF0EE3CFEAFFE9CFF3FF1D
:102BC000EACFF4FF0900F5CFEFFFEE66FBD7120066
:102BD000FE0EE3CFE9FFFF0EE3CFEAFFF36AF46AEC
:0C2BE000EE5203E0F34AF42AFBD7120087
:042BEC001B6A1A6ADC
:102BF000196A186A200EE76ED8901C361D361E36EC
:102C00001F36183619361A361B362150185C2250DA
:102C1000195823501A5824501B5809E32150185EA4
:102C20002250195A23501A5A24501B5A1C2AE72E94
:042C3000E4D71200D3
:0C2C3400D9CFE6FFDACFE6FFE1CFD9FFF1
:102C4000E2CFDAFFE652F20E0001E417ABAC03D09C
:102C5000E491ABB0E481ABB4E485ABB2E487AE50B1
:102C6000DF6EDF50E552E552E5CFDAFFE7CFD9FF5F
:022C7000120050
:0E2C7200D9CFE6FFDACFE6FFE1CFD9FFE2CF00
:102C8000DAFFE652E652FC0EDBCFDEFFDBCFDDFFE4
:102C9000010EDB50B36EDF50B26EE552E552E552E5
:0A2CA000E5CFDAFFE7CFD9FF1200FD
:062CAA00D9CFE6FFDACFEE
:102CB000E6FFE1CFD9FFE2CFDAFFE652E652FC0EA3
:102CC000DBCFDEFFDBCFDDFF010EDB50CF6EDF5051
:102CD000CE6EE552E552E552E5CFDAFFE7CFD9FFF8
:022CE0001200E0
:0E2CE200D9CFE6FFDACFE6FFE1CFD9FFE2CF90
:102CF000DAFFACAC04D0AC900001E4B3AC80FD0EC4
:102D0000DB50AD6EE552E5CFDAFFE7CFD9FF120019
:102D1000000EF36E00EE00F0060E01D81200EA601D
:102D200002D0EE6AFCD7F350E9601200EE6AFCD7DD
:102D300015EE00F025EE00F0F86A279C48EC15F03F
:0C2D400003EC00F048EC09F0FBD7120097
:042D4C0031384632A2
:102D500035325F4361706163696D5F43413535357D
:102D60005F706F6F6C696E672E630D0A202073743D
:102D700072696E6720656E2052414D0D00000000A3
:102D800000000000000000000000000000013030E2
:102D90003030303030300031323334353637383936
:102DA0003031323334350004303030303030303070
:102DB0003030303030303030303030303030300043
:102DC00004040404040404040404040404040404C3
:102DD00004040404040404040404040404040404B3
:102DE0000404040404040404B028B428CE280429EC
:102DF0003D295B299029B429C529D629E729F82935
:102E0000092A1A2A2B2A362A412A522A632A742A84
:082E1000792A7E2AB3150100A6
:020000040030CA
:01000100FA04
:01000200F409
:01000300FEFE
:01000600FBFE
:00000001FF
